:020000040000FA
:020000001728BF
:08000800C000030EC1000B1B38
:100010000C1C0D28A5200C1012288B1A0B1D122861
:10002000AF200B11410E8300C00E400E0900831655
:10003000FF2390008312203084008001840A041F73
:100040001D28841E1D288316810196018C019901AB
:1000500083120730990090018316850185160516D5
:100060009501951615168B018B170B178C010C1427
:1000700083128510851A44288D208D20992099207F
:10008000992099208D204928051A3A288D209920F9
:100090005B28851E56288420851E56288D20992091
:1000A0008D2099209920992099203A28051A4928CD
:1000B00099208D206E28851A6728992099208D20F7
:1000C000992099209920992099208D206E28051E2D
:1000D0005B288420051E5B2899203A28851E7D28F0
:1000E0008420851E7D28992099208D208D208D20AB
:1000F0008D208D208D2099205B28051E6E28842060
:10010000051E6E288D204928C830A300FA30A400AF
:10011000A40B8828A30B86280800FD30A1008F00BF
:100120001B30A2008E001014FF30A000101896287B
:100130000800FA30A1008F00C930A2008E00101410
:10014000FF30A0001018A2280800101021088F000E
:1001500022088E0002308506A00B1014080008004B
:02400E00843FED
:00000001FF
